:100000000BC018951895189518951895189518956A
:1000100018951895189518958FED8DBFC0ECE4EBE9
:100020004E2EDD275D2EEEE7F0E0A0E6B0E0A895CD
:1000300084B7082E877F84BF88E1992781BD91BD51
:1000400088278D933197E9F7A5D166248DEF8ABB78
:100050008FED87BB80E08BBB80E088BBD99A83E8BB
:1000600086B980E087B97CD18CE0DCD1E2EAF7E0A8
:100070006FD1E2E0F0E085D180E080936700EEE0B0
:10008000F0E0A3E691E072D3009163000E3C08F02B
:1000900005C085B78F7E806385BF8895A4E63FD372
:1000A00080E08093660080E080936200ABE637D307
:1000B000809171008F778093710052D1E2EBF7E06D
:1000C00047D1D198A1E79C9196FF04C0C99B0EC06F
:1000D0009F7B9C93C9990AC084E69F939927CED1B0
:1000E0009F91C99903C090649C93F7D0379AEF937E
:1000F000FF93E5E1F0E0B6D1FF91EF9107B1007E0B
:10010000086007B9CAD1ABE68D939C933798EBE6AC
:10011000F0E0D190E080FF2400272AD2ADE659D24A
:10012000EAE9F7E0F3D2EDE6F0E0FED164D2EDE0EB
:10013000ADE6FDD2EEE9F7E0E9D2EDE6F0E0F4D18C
:1001400093D2EDE0B3D1A1E6DC92A1E60C914AE0B6
:1001500014D30C9300916100003010F009F001C03D
:1001600001C02DD084E690E089D100916600063070
:1001700009F023C0A1E78C9187FB0EF010C0EAE0E4
:10018000F0E0A4E67BE7E0D2EBD0E0ECF7E0E0D0F3
:1001900060D0809171008F778093710070CFEAE01A
:1001A000F0E0A4E1E2D2A4E60D911C91041715073A
:1001B00009F002C075C001C030C083CF54CFD89AB7
:1001C00084E690E05BD1D89884E690E057D1A6E62B
:1001D0008C918F5F8C930091660045E0040FA2E63E
:1001E0000C938FEBA2E61C91CAD0EEECF7E0B0D0F6
:1001F000A4E60D911C914AE050E097D0A4E60D933F
:100200001C93A4E60D911C91A1E64D915527040F76
:10021000151FA4E60D931C930895A2D0E0EDF7E01E
:1002200097D0A7E68C918F5F8C9389E080936800CC
:100230008FE58093690015D000916700033009F0C5
:1002400007C0ECE3F0E09DD080E08093670001D030
:1002500016CF82E08093680088EC8093690001D01B
:10026000089584E690E00AD181E080936A0040918D
:10027000680000916A00041710F009F010C0D89AC5
:10028000A9E68C919927FAD0D898A9E68C9199275C
:10029000F5D0AAE68C918F5F8C9308F4E8CF08958F
:1002A0005FD0EEEDF7E054D0D4DF58D0EEEEF7E0BB
:1002B0004FD08CE291E0E2D0DA9AE2E0F0E061D057
:1002C000DA9880916300815080936300EEE0F0E063
:1002D000A3E691E07BE739D2D2CE809171008068AD
:1002E00080937100B6DF089504D01FD000FC0CD0BD
:1002F00008950024E89457FF02C009D0689400F8DC
:100300000BD010F80124089502D009D0089550951B
:1003100040954F5F5F4F0895E89417FF089500954B
:1003200010950F5F1F4F68940895752F642F552700
:100330004427FF93F1E1889405C010F4460F571F3E
:100340005695479517950795FA95B9F7FF91089532
:10035000D9D1802D11F060D0FBCF089580EC62C020
:1003600081E060D014D080E85DC08FE7213039F0A3
:100370008FEB223021F08FE8233009F08FEC810FD2
:1003800051C088EE93E07AD03197D9F7089583E091
:10039000992774C08AEF90E071D0B89AB99ABA9A46
:1003A000BB9AD49AD59ADD9885E090E067D0DC9826
:1003B000C098C198C29AC39ADC9AEF93FF93E5E183
:1003C000F0E050D0FF91EF91DC9855D0DC9AEF939C
:1003D000FF93E5E1F0E046D0FF91EF91DC984BD040
:1003E000DC9AEF93FF93E5E1F0E03CD0FF91EF91D1
:1003F000DC9841D0C398DC9AEF93FF93E5E1F0E0FD
:1004000031D0FF91EF91DC9836D088E20BD08EE0AE
:1004100009D086E007D00895DD9A829505D004D0F2
:100420002AD00895DD98F9CF859510F4C39A01C0BC
:10043000C398859510F4C29A01C0C298859510F4AE
:10044000C19A01C0C198859510F4C09A01C0C098A6
:10045000DC9AEF93FF93E5E1F0E004D0FF91EF9198
:10046000DC9808953197F1F70895689462F808953B
:10047000E89462F8089581E090E000C0EF93FF9364
:10048000EE27E82BE92B31F0EAEFF0E03197F1F7B6
:100490000197D1F7FF91EF910895369A3699FECFE3
:1004A000369A3699FECF84B195B108953DD09927FB
:1004B00011278F2D880F80E8F82A802F881F08F4D5
:1004C0001FEF41F08F57082F07FD04C0003240F0A6
:1004D0008FEF01C08827982FD82EE82EF82E09C05C
:1004E0008FE1801B082FF694E794D79497950A958F
:1004F000D1F7112351F09095D094E094F09481E0DD
:10050000980F8827D81EE81EF81E0F2DFE2CED2C04
:10051000D92E0895D094E094F09491E0D90E9927C3
:10052000E91EF91E10950895D190E190F190019186
:10053000089521913191419151910895102F90E8A2
:10054000FF0C001F0927990FF7941078652F90E88A
:10055000440F551F5927990F479560780038089523
:10056000FF0C90E89027110F9795F794092F0895A5
:10057000102FBD2CDE2CEF2CF02E11234AF4B0945A
:10058000D094E094F0949FEFB91AD90AE90AF90AD5
:100590000EE1FF2039F4FE2CED2CDB2CBB2408509F
:1005A000C2F723C032F00A95BB0CDD1CEE1CFF1C09
:1005B000F9CF01D0D5CFB7FE089590E8B91611F460
:1005C000D0FE08959FEFD91AE90AF90A09F40395B4
:1005D0000895DD92ED92FD920C9308959FE7092F07
:1005E000F92A9FEFD92EE92E0895DD24EE24FF2469
:1005F000002711270895A2DFC1F35038B1F3162761
:10060000005850580894051F12F418F4E7CF08F06A
:10061000ECCF0AD0FF202AF0BB0CDD1CEE1CFF1C27
:100620009FCF0F5FDBF29CCF9F929924AA24BB241B
:10063000992788E1990CAA1CBB1CDD1CEE1CFF1C31
:1006400030F4920EA31EB41ED91EE91EF91E8A951F
:1006500089F79F9008950AF045D082CF5FE3222763
:100660003327442701C065DF69DF5038B1F3003814
:1006700099F3902F951B8BF312F434D0FACF983165
:1006800018F0222733274427983028F0232F342FBF
:1006900044279850F9CF992329F046953795279507
:1006A0009A95D9F7912F962742F014D0B0F6F79487
:1006B000E794D7940F5F8BF691CF10D051F008F4E8
:1006C00029DFFF2052F2DD0CEE1CFF1C0150CBF79E
:1006D00085CF8BCFD20EE31EF41E0895D21AE30A03
:1006E000F40A0895DF92EF92FF920F931F93D22E98
:1006F000E32EF42E052F162F6F915F914F913F91AE
:100700002F910895C895319600200895FBDF202D84
:10071000F9DF302DF7DF402DF5DF502D089582E011
:1007200001C084E099279D938A95E9F7089594E0A4
:1007300081918D939A95E1F70895E199FECFEEBBF3
:100740003196089591E001C092E07B3751F47FB774
:10075000F894F3DF8D918DBBE29AE19A9A95C9F7EF
:100760007FBF7727089591E001C092E0E6DFE09A2D
:100770008DB38D939A95D1F70895FF93881BF9E077
:10078000001FFA9511F4FF910895881F841B18F437
:10079000840F8894F5CF0894F3CF8FC2F53D000005
:1007A000A0405757572E4156522E344D472E434F97
:1007B0004D00202020456E74657220636F646500D3
:1007C0002020436F64652073746F726564002A0093
:1007D000202020436F64652077726F6E670020438E
:1007E0006F64652061636365707465640000202038
:0C07F0002020556E6C6F636B6564000088
:00000001FF
